:1000000000308A0012280000103084000008031914
:1000100011280F2800000000000000000000800BE5
:100020000A28003484011F30830508308C008C1DA1
:10003000212807308101813084000008C0390F3841
:1000400080006400813084000008C0390C04800006
:1000500083160610831206148316051183120511E8
:1000600083168511831285118316861283128612D8
:100070008316861183128615C7308C008C0B3E28A0
:1000800000000000831686118312861183168511E5
:10009000831285150C308F00FA30900004208F0BEE
:1000A0004C28831686128312861628308F00FA3069
:1000B000900004208F0B5728831686128312861215
:1000C0008316051183120515C8309000042083168D
:1000D00085118312851104308F00FA3090000420BE
:1000E0008F0B6D288316851183128515C8309000FB
:1000F0000420831685118312851104308F00FA3095
:10010000900004208F0B7F28831686128312861698
:10011000C8309000042083168612831286120430A1
:100120008F00FA30900004208F0B912883168612DE
:1001300083128616C830900004208316861283121C
:1001400086128316051183120511831685118312F9
:100150008511831686128312861283160610831267
:040160000610630022
:02400E00F03F81
:00000001FF
